:100000000C947B030C94BF030C94BF030C94BF03AC
:100010000C94BF030C94BF030C94BF030C94BF0358
:100020000C94BF030C94BF030C94E80F0C94BA100B
:100030000C94BF030C94BF030C94BF030C94BF0338
:100040000C94BF030C94C4240C94BF030C94BF0302
:100050000C94BF030C94571E0C94BF030C94BF0365
:100060000C94BF030C94BF030C94BF030C94BF0308
:100070000C94BF030C94BF030C94BF030C94BF03F8
:100080000C94BF030C94BF030C94BF030C94BF03E8
:100090000C94BF030C94BF030C94BF030C94BF03D8
:1000A0000C94BF030C94BF030C94BF032711491198
:1000B0003712491137128E11B11137120612191267
:1000C000E814E814171517154D156D159E169E1694
:1000D00078159E16281628168F169E169E169816A8
:1000E00035163516351635163516351635163516B8
:1000F00035163516351635163516351635163516A8
:10010000471654165B1662166C160122022201C4B1
:1001100002C4000121022101C402C4000120022006
:1001200001C402C400011F021F01C402C400013146
:10013000023101C402C40001E10131023102E101D6
:10014000C402C4000126022601C402C40001250223
:100150002501C402C4000124022401C402C4000118
:1001600023022301C402C40001E10134023402E18C
:1001700001C402C400012D022D01C402C40001E12A
:100180000127022702E101C402C40001E1012502A6
:100190002502E101C402C400011E021E01C402C402
:1001A0000001E10130023002E101C402C40001E1BA
:1001B000012F022F02E101C402C40001270227011E
:1001C000C402C400012E022E01C402C40001E101D8
:1001D00026022602E101C402C4000138023801C42B
:1001E00002C40001E1011E021E02E101C402C400BA
:1001F0000130023001C402C400012F022F01C402E9
:10020000C40001E1012D022D02E101C402C400017C
:10021000E10121022102E101C402C40001E1011F48
:10022000021F02E101C402C40001E1012E022E02FC
:10023000E101C402C40001E10138023802E101C455
:1002400002C40001E10124022402E101C402C4004D
:1002500001E10122022202E101C402C4000000F017
:10026000A101840884088A35002B00297FE1000061
:100270000000001E00140004001D0000004D001FBF
:1002800000070016001B00E0002C00200015000BEA
:10029000001000E2002A0021001A0017000600E307
:1002A000004A00220005000A00190000000000506A
:1002B00000015400000000000000004F0001540045
:1002C0000000770000000023000D001C000E00005D
:1002D0000000002400090011000F0050004B002511
:1002E00000180008003600510028002600130012F4
:1002F00000370052002C00270033000C0038714FEB
:10030000004E002D0031003400E500C40000000163
:1003100000010001000100010000003A0022023843
:10032000002300010001003B0024022602240001FA
:100330000001003C0038022E002500010001003DB4
:10034000002E0227002600010001003E001F022FA0
:100350000231020000010001000100000001000064
:100360000001000100010000000100000001003F49
:10037000002102300238000000010040002D021E62
:10038000001F000100010041002F00250220000194
:10039000000100420030002702210001000100435B
:1003A000001E022D0022000100010044004500341F
:1003B0000001000100000001000100010001000136
:1003C0000000000100010001000100010001000126
:1003D000000100F2000100010001000100F000F145
:1003E000000100F400010001000100F3000100F52C
:1003F00000010001000100010001000000010001F6
:1004000000010000000100000001000100010000E7
:1004100000010000000100010001000100010000D6
:100420000001000100010001000100A9000100011C
:100430000001000100AC00AA00B6000100010001AB
:1004400000AB00A800010001000100010001000153
:1004500000010001000100AE0001000100000001E8
:1004600000010001000100010000003A0064306D4D
:10047000307830010001003B0065306E307930018A
:100480000001003C0066306F307A30010001003D11
:1004900000673070307B30010001003E0068307131
:1004A000307C30000001000100010000000100006C
:1004B0000001000100010000000100000001003FF8
:1004C00000693072307D300000010040006A3073F6
:1004D000307E300100010041006B3074307F30010C
:1004E00000010042006C3075308030010001004393
:1004F00000823076308130010001004400450077F1
:100500003001000100000016034500720067006F13
:100510000044006F007800200045005A00000016DB
:10052000034500720067006F0044006F00780020F0
:100530000045005A0000000403090409026D00048C
:100540000100A0FA090400000103010100092111C2
:10055000010001223F000705810308000A09040188
:10056000000103010200092111010001224D0007D1
:1005700005820308000A09040200010300000009C3
:1005800021110100012236000705830308000A0932
:1005900004030001030000000921110100012239B8
:1005A000000705840310000112011001000000087B
:1005B000EDFE071301000102000105010906A1017A
:1005C000050719E029E71500250195087501810245
:1005D0000508190129059505750191029501750315
:1005E00091010507190029771500250195787501F6
:1005F0008102C005010980A101850216010026B70C
:10060000001A01002AB700751095018100C0050C81
:100610000901A1018503160100269C021A01002A86
:100620009C02751095018100C005010902A1010914
:1006300001A1000509190129051500250195057578
:100640000181029501750381010501093009311508
:1006500081257F95027508810609381581257F95CA
:100660000175088106050C0A38021581257F950160
:1006700075088106C0C005010906A101050719E03A
:1006800029E7150025019508750181029501750876
:10069000810105081901290595057501910295014A
:1006A000750391010507190029FF150025FF95061F
:1006B00075088100C000000000000000000000007C
:1006C000010204060A0F17202C3A4A5D71879DB378
:1006D000C7DAE9F5FCFFFCF5E9DAC7B39D87715D80
:1006E0004A3A2C20170F0A060402010000000000FD
:1006F00000000000000011241FBECFEFDAE0DEBFD3
:10070000CDBF04B603FE24C08091FB019091FC0193
:10071000A091FD01B091FE018730904BA740B04BF6
:10072000B9F41092FB011092FC011092FD0110929D
:10073000FE0114BE84B7877F84BF88E10FB6F894AA
:1007400080936000109260000FBEE0E0FFE3099527
:1007500011E0A0E0B1E0E6E1FDE402C005900D92F9
:10076000A433B107D9F711E0A4E3B1E001C01D92B1
:10077000AB3FB107E1F70E942C0D0C9489260C9435
:1007800000001092B9008AE08093B800089594EABE
:100790009093BC009091BC0097FFFCCF9091B90062
:1007A000987F983021F0903111F081E00895809386
:1007B000BB0084E88093BC008091BC0087FFFCCF25
:1007C0008091B900887F883111F0803471F780E022
:1007D000089584E98093BC008091BC0084FDFCCF27
:1007E00008958093BB0084E88093BC008091BC0096
:1007F00087FFFCCF9091B900987F81E0983209F48F
:1008000080E0089584E88093BC008091BC0087FF5D
:10081000FCCF8091BB00089580910101811115C02A
:1008200080E40E94C7038093010181110CC082E122
:100830000E94F10380930101811105C08FEF0E9496
:10084000F103809301010E94E90384B1807F84B9A0
:1008500085B1807F85B98AB1837F8AB98BB1837F67
:100860008BB93E98469808950E94C7058093010170
:100870000E940C0480B38C7080BB81B3836F81BBFA
:10088000A5E3B1E0E3E4F1E08EE08E0F11921D925A
:100890008E13FCCF0C94B105BF92CF92DF92EF92F2
:1008A000FF920F931F93CF93DF93809101018823D1
:1008B00079F0809134018F5F80933401811108C0F9
:1008C0000E94C70580930101811102C00E94590551
:1008D00005E311E0C0E0D0E0DD24D39482E0C82E2F
:1008E000EE24E394F12CC730D10500F5809101018D
:1008F000811164C080E40E94C703809301018111CB
:1009000012C082E10E94F1038093010181110BC0AA
:10091000C7010C2E01C0880F0A94EAF780950E9447
:10092000F103809301010E94E90348C0CA30A1F09D
:1009300028F4C83059F0C93061F005C0CC3089F0D6
:1009400070F0CD3089F0209A289810C0219A29980B
:100950000DC0229A2A980AC0239A2B9807C0529A4F
:1009600001C0539A5B9802C03E9A469890EA9A95C5
:10097000F1F79FB1799902C082E001C080E09170E7
:100980009D25982B7C9902C084E001C080E0892BD2
:100990007D9902C038E001C030E0832B7E9902C00F
:1009A00020E101C020E0822B9FB19095991F9927EB
:1009B000991F9295990F907E892B0FC0809101010C
:1009C000811149C080E40E94C703809301018823FC
:1009D00079F1B12C0E94E9038B2DF80190819817D1
:1009E00019F08083C09200010E940C0421960F5FD1
:1009F0001F4FCE30D10509F076CF809100018823BA
:100A000061F1815080930001882339F08FE99FE0E4
:100A10000197F1F700C0000020C0A3E4B1E0E5E3D6
:100A2000F1E0CF01825F91919D938E13FCCF15C0B1
:100A300083E10E94F103809301018111CACF81E417
:100A40000E94C703809301018111C3CF0E94020459
:100A5000B82EB094BFCF80E0C0CF0E94570581E090
:100A6000DF91CF911F910F91FF90EF90DF90CF908A
:100A7000BF900895E82FF0E0ED5BFE4F8081089570
:100A800008950F931F93CF93DF93C3E4D1E010E059
:100A90000C2F025F899190E00E947D1D180F0C13AE
:100AA000F9CF812FDF91CF911F910F9108950C9471
:100AB000AC0756985E9825982D9826982E982798DA
:100AC0002F988FEF90E09093890080938800909307
:100AD0008B0080938A0090938D0080938C00259AE0
:100AE0002D9A2FEF80E792E0215080409040E1F76F
:100AF00000C00000269A2E9A2FEF80E792E0215046
:100B000080409040E1F700C00000279A2F9A2FEF15
:100B100080E792E0215080409040E1F700C0000063
:100B200025982D982FEF80E792E02150804090404B
:100B3000E1F700C0000026982E982FEF80E792E0A2
:100B4000215080409040E1F700C0000027982F9886
:100B500056985E9825982D9826982E9827982F9825
:100B6000089589EA8093800089E080938100249829
:100B70002C983F988AB18F748AB96E98479A8BB136
:100B8000806B8BB9769A0E9459050C94AB0780E272
:100B9000809301018091510181110EC00E94C10317
:100BA00081E0809351012FEF83ED90E3215080404D
:100BB0009040E1F700C0000080E40E94C7038093EA
:100BC000010181112EC00E94F10380930101811166
:100BD00028C00E94F10380930101811122C08FE39C
:100BE0000E94F1038093010181111BC00E94E9035F
:100BF00080E40E94C70380930101811112C08CE040
:100C00000E94F1038093010181110BC00E94F10346
:100C100080930101811105C08FE30E94F10380934D
:100C200001010E94E903809101010895CF93DF93B0
:100C3000EC01623709F4C6C038F56A3609F483C09E
:100C400098F4663609F463C048F4643609F451C078
:100C500008F056C0662309F441C01AC1683609F489
:100C600064C008F45BC068C06E3609F48FC030F40D
:100C70006C3609F476C008F46DC081C0603709F4A1
:100C800093C008F48AC097C06A3709F4D0C080F4D2
:100C9000663709F4B3C030F4643709F4A1C008F42E
:100CA00098C0A5C0683709F4B6C008F4AEC0B9C092
:100CB0006E3709F4D4C030F46C3709F4C4C008F4BA
:100CC000BCC0C7C0603809F4D6C008F4CEC06138D3
:100CD00009F4D7C0623809F44BC0DAC08A8188238E
:100CE00021F085EE0E948C13D2C085EE0E94541430
:100CF000CEC00E94271B8A81882309F4C9C0CBC0BB
:100D00000E94271B8A81882309F4C2C0C7C00E94A1
:100D1000271B8A81882309F4BBC0C3C00E94271BFC
:100D20008A81882309F4B4C0BFC00E94271B8A812E
:100D3000882309F4ADC0BBC00E94271B8A81882389
:100D400009F4A6C0B7C00E94271B8A81882309F432
:100D50009FC0B3C00E94271B8A81882309F498C0D2
:100D6000AFC00E94271B8A81882309F491C0ABC0C1
:100D70000E94271B8A81882309F48AC0A7C00E9489
:100D8000271B8A81882309F483C0A3C00E94271BE4
:100D90008A81882309F47CC09FC00E94271B8A8116
:100DA000882309F475C09BC00E94271B8A81882371
:100DB00009F46EC097C00E94271B8A81882309F41A
:100DC00067C093C00E94271B8A81882309F460C0F2
:100DD0008FC00E94271B8A81882309F459C08BC0C9
:100DE0000E94271B8A81882309F452C087C00E9471
:100DF000271B8A81882309F44BC083C00E94271BCC
:100E00008A81882309F444C07FC00E94271B8A81FD
:100E10008823F1F17CC00E94271B8A818823C1F1BD
:100E200079C00E94271B8A81882391F176C00E9495
:100E3000271B8A81882361F173C00E94271B8A8146
:100E4000882331F170C00E94271B8A81882301F119
:100E50006DC00E94271B8A818823D1F06AC00E943E
:100E6000271B8A818823A1F067C00E94271B8A81E3
:100E7000882371F064C00E94271B8A81882341F077
:100E800061C00E94271B8A81882311F05EC060C068
:100E900020E030E05CC020E532E059C023E432E0DD
:100EA00056C026E332E053C029E232E050C02CE1C4
:100EB00032E04DC02FE032E04AC022E032E047C0CD
:100EC00029EF31E044C020EF31E041C023EE31E0B2
:100ED0003EC02AED31E03BC02DEC31E038C024ECBF
:100EE00031E035C02BEB31E032C02EEA31E02FC0CB
:100EF00021EA31E02CC028E931E029C02BE831E0BB
:100F000026C02EE731E023C025E731E020C028E6E7
:100F100031E01DC02FE531E01AC026E531E017C0F1
:100F20002DE431E014C024E431E011C027E331E0C6
:100F30000EC02EE231E00BC025E231E008C02CE10A
:100F400031E005C023E131E002C02AE031E0C9010F
:100F5000DF91CF91089508956091BD017091BE0118
:100F60008091BF019091C0010E94891D56985E98A2
:100F700025982D9826982E9827982F98813019F02B
:100F8000823021F00895259A2D9A0895269A2E9A56
:100F9000089581E0089581E008950C94CB070895A9
:100FA0000F931F93CF93DF938C01FC01C081D181FC
:100FB000CE010E94021CBE010E947908EC01B8011A
:100FC0000E94CD07882309F48DC0F801828188230F
:100FD00009F44AC080915D0181111FC0C431F0E560
:100FE000DF0709F051C00E94CF0781E080935D01C7
:100FF0000E94211E90935C0180935B01109254012A
:1010000010925601109255011092580110925701FA
:1010100010925A011092590165C080915B01909124
:101020005C010E942D1E883C910570F48091540152
:10103000E82FF0E0EE0FFF1FEB5AFE4FD183C08385
:101040008F5F809354014EC0C43880E5D80721F0EB
:10105000C538D04501F13AC0F8018281882341F0BA
:101060001092520182E01EC0C438E0E5DE0759F557
:1010700080915201811106C086E20E948C1386E2A3
:101080000E94541482E01CC0C438F0E5DF0741F32D
:10109000C538D045D9F4F8018281882331F0109207
:1010A000530180E20E94A3141DC08091530181115D
:1010B00006C087E20E948C1387E20E94541480E2EB
:1010C0000E94AA140FC0C538D04529F381E080934F
:1010D000520180935301C801DF91CF911F910F916D
:1010E0000C94C90780E0DF91CF911F910F91089573
:1010F000089596E0799FF001112494E5899FE00D11
:10110000F11D1124E60FF11DEE0FFF1FE959FD4FF0
:10111000859194910895880F991FFC01E352FF4F28
:10112000859194910895880F991FFC01E35AFD4F12
:101130008591949108950F931F93CF93DF93EC01C2
:10114000811520E3920750F5C11580E2D80708F019
:10115000C3C0CB3BD10590F4C83AD10508F06AC0B2
:10116000C53AD10508F05BC0C430D10508F0D0C144
:10117000219709F0CAC101E010E00AC2CF3FD105B2
:1011800011F008F0C5C1C03FD10508F0A2C0CE01E2
:10119000805E9109089708F4BBC1B7C1C13090E5E2
:1011A000D90709F4A2C020F5C0318FE4D80770F444
:1011B000C11590E4D90708F094C0C11521E3D20706
:1011C00008F0A3C1DD278E01106CE2C1C115D04526
:1011D00009F09BC10E9409178FEF94E32CE0815026
:1011E00090402040E1F700C000000E947C1ED0C16A
:1011F000C11597E5D90758F4C03121E5D20708F0A9
:101200001CC1C43180E5D80708F475C07EC1CE0189
:1012100090578115904108F078C1DF7073C1C53ACD
:10122000D10509F477C1C63AD10509F076C102E8C3
:1012300010E4AEC1C83AD10509F472C1C93AD1056A
:1012400009F471C1CA3AD10509F470C1CB3AD1058C
:1012500009F46FC1CC3AD10509F46EC1CD3AD1057C
:1012600009F46DC1C03BD10509F46CC1CE3AD1057A
:1012700009F46BC1CF3AD10509F46AC1C13BD1056C
:1012800009F469C1C23BD10509F468C1C33BD1056A
:1012900009F467C1C43BD10509F466C1C53BD1055A
:1012A00009F465C1C63BD10509F464C1C73BD1054A
:1012B00009F463C1C83BD10509F462C1C93BD1053A
:1012C00009F461C1CA3BD10509F460C100E014E42E
:1012D0005FC18E0110655CC1CE019F700E949308B2
:1012E00058C1DF708E01106A53C18091DA018160AC
:1012F0008093DA014DC10E942120811102C00E9419
:1013000007200E943E2090E09093FB018093FA0119
:10131000C23080E5D80721F48091FA01816086C04F
:10132000C43090E5D90721F48091FA0182607EC033
:10133000C63020E5D20721F48091FA01846076C09E
:10134000C83080E5D80719F48091FA0127C0CA3067
:1013500090E5D90721F48091FA01806167C0CC3013
:1013600020E5D20721F48091FA0180625FC0CE307F
:1013700080E5D80721F48091FA01806457C0C0311C
:1013800090E5D90721F48091FA0180684FC0C231FD
:1013900020E5D20729F48091FA018460886046C074
:1013A000C33080E5D80721F48091FA018E7F3EC0DA
:1013B000C53090E5D90721F48091FA018D7F36C0C0
:1013C000C73020E5D20721F48091FA018B7F2EC02F
:1013D000C93080E5D80719F48091FA0126C0CB30D6
:1013E00090E5D90721F48091FA018F7E1FC0CD309E
:1013F00020E5D20721F48091FA018F7D17C0CF300C
:1014000080E5D80721F48091FA018F7B0FC0C131AC
:1014100090E5D90721F48091FA018F7707C0C33195
:10142000D04531F48091FA018B7F877F8093FA0158
:101430008091FA010E944220ABC08D2F99278F70B6
:10144000992781309105D9F49E012370332702C07A
:10145000880F991F2A95E2F79C688E0144E0000FDF
:10146000111F4A95E1F700271370802B912B53E051
:10147000CC0FDD1F5A95E1F7C076DD272FC08230F3
:10148000910531F4DC2FCC278E01016F106A80C0EA
:101490008330910569F4CE018370992701E010E053
:1014A00002C0000F111F8A95E2F7C8019C680FC0A7
:1014B00084309105B9F4CE018370992701E010E0E2
:1014C00002C0000F111F8A95E2F7C8019A6823E055
:1014D000CC0FDD1F2A95E1F7C07ED7708C010C2B55
:1014E0001D2B56C08530910531F4DC2FCC278E01A1
:1014F000046F106A4DC0069709F04AC0CF71DD270E
:10150000DC2FCC278E01106243C000E010E040C009
:101510008E013EC001E810E43BC003E810E438C08F
:1015200002EE14E435C009EE14E432C00AEE14E40D
:101530002FC005EB14E42CC006EB14E429C007EB24
:1015400014E426C00CEC14E423C00DEC14E420C019
:1015500003E815E41DC00AE815E41AC002E915E421
:1015600017C004E915E414C001E216E411C003E257
:1015700016E40EC004E216E40BC005E216E408C04F
:1015800006E216E405C007E216E402C00AE216E429
:10159000C801DF91CF911F910F91089596E0799F37
:1015A000F001112494E5899FE00DF11D1124E60F4F
:1015B000F11DEE0FFF1FE959FD4F85919491803E7B
:1015C0009105E0F4803C910558F58133910509F4CB
:1015D0006FC048F48932910509F463C08A329105DD
:1015E00009F46DC072C089339105E9F08238910524
:1015F000D1F08533910509F44DC067C0833E910554
:1016000081F138F4803E9105B9F0823E9105D9F020
:101610005CC0863E910561F1873E9105A1F155C000
:101620000E948B0808952091FA0120FD02C021FF3D
:101630004CC080EE90E049C08091FA0180FFF9CF64
:1016400089E390E042C08091FA0182FF0EC0809150
:10165000FA0184FF03C080E090E037C083EE90E0A1
:1016600034C08091FA0182FFF2CF82EE90E02DC06B
:101670008091FA0183FF0BC08091FA0184FDEBCFCA
:1016800087EE90E022C08091FA0183FFF5CF86EECD
:1016900090E01BC08091FA0185FF07C089E290E0CD
:1016A00014C08091FA0185FFF9CF85E390E00DC069
:1016B0008091FA0186FF07C08AE290E006C080911F
:1016C000FA0186FFF9CF81E390E00E949B0808951C
:1016D00008950C94680B80916E010895CF93DF9369
:1016E00000D01F92CDB7DEB79C018091F10184300C
:1016F00019F593E099833B832A839093E9008FEF58
:101700009091E800815095FD06C095ED9A95F1F70E
:1017100000008111F5CF8091E80085FF0DC040E009
:1017200050E063E070E0CE0101960E94D80D8091F8
:10173000E8008E778093E8000F900F900F90DF9174
:10174000CF910895CF93DF9300D01F92CDB7DEB72E
:101750002091F101243021F522E029839B838A83A3
:1017600083E08093E9008FEF9091E800815095FD30
:1017700006C095ED9A95F1F700008111F5CF8091A3
:10178000E80085FF0DC040E050E063E070E0CE016E
:1017900001960E94D80D8091E8008E778093E80032
:1017A0000F900F900F90DF91CF9108952091F1014C
:1017B0002430F1F422E02093E9002FEF3091E8008B
:1017C000215035FD06C035ED3A95F1F700002111A5
:1017D000F5CF2091E80025FF0BC040E050E065E028
:1017E00070E00E94D80D8091E8008E778093E80029
:1017F0000895CF93DF93EC019091F101943009F0BB
:1018000046C080910C018823D9F080910D01882376
:10181000B9F09093E9008FEF9091E800815095FD29
:1018200006C095E19A95F1F700008111F5CF8091FE
:10183000E80085FF2CC040E050E060E170E017C098
:1018400081E08093E9008FEF9091E800815095FD51
:1018500006C095ED9A95F1F700008111F5CF8091C2
:10186000E80085FF14C040E050E068E070E0CE0181
:101870000E94D80D8091E8008E778093E80080E187
:10188000FE01AEE5B1E001900D928A95E1F7DF919E
:10189000CF9108958091F001811109C00E946D0FD0
:1018A0000E94CA0F8091E20084608093E200089554
:1018B0001092F001089508950C94B1240E94121E14
:1018C0000E94B7240E9470120C94690B42E061ECF4
:1018D00081E00E94E70E42E061EC82E00E94E70EA8
:1018E00042E061EC83E00E94E70E42E161EC84E0BB
:1018F0000C94E70E8091F301833009F455C030F465
:10190000813071F0823009F48EC008958A3009F474
:101910007AC08B3009F460C0893009F09CC020C0C7
:101920008091F201813A09F096C08091E800877FAA
:101930008093E8008091F6019091F701892B21F4C2
:1019400060E18EE591E003C060E080E090E070E04F
:101950000E94230E8091E8008B778093E800089521
:101960008091F201813209F076C08091F601909168
:10197000F701009719F0039709F06DC08091E80016
:10198000877F8093E8008091E80082FD05C0809108
:10199000F1018111F8CF5FC08091F10080936E0159
:1019A0008091E8008B7753C08091F201813A09F071
:1019B00052C08091F6019091F701892B09F04BC03C
:1019C0008091E800877F8093E8008091E80080FFA5
:1019D000FCCF80910C0136C08091F2018132D9F5A3
:1019E0008091F6019091F701892BA9F58091E8008B
:1019F000877F8093E8000E941C0F8091F401809300
:101A00000C010C9409178091F201813221F580912B
:101A1000E800877F8093E8000E941C0F8091F50109
:101A200080936F0108958091F201813AA1F4809131
:101A3000E800877F8093E8008091E80080FFFCCF7A
:101A400080916F018093F1008091E8008E77809300
:101A5000E8000C941C0F089584B7877F84BF88E149
:101A60000FB6F89480936000109260000FBE90E073
:101A700080E80FB6F89480936100909361000FBEE8
:101A80000E94BF120E946D0F0E94CA0F8091E20057
:101A900084608093E20078940E9450120E94C112E8
:101AA00082E091E00E946B120E949F248091F101DC
:101AB000853069F40E94D91D8091EF018823B1F32C
:101AC0000E94041E882391F30E94C20DEFCF0E9452
:101AD000C712ECCF292F332723303105C9F064F426
:101AE0002130310581F02230310509F043C08DE607
:101AF00090E02BE335E042C021323105F1F0223293
:101B0000310541F137C082E190E028EA35E036C086
:101B100099278130910541F08230910541F0892B60
:101B200049F5E7E3F5E005C0EFE1F5E002C0E7E0E5
:101B3000F5E0849190E09F0121C06430D8F4E62F55
:101B4000F0E0EE0FFF1FEE5DFE4F2081318189E056
:101B500090E014C0643070F470E0FB01EE0FFF1FE2
:101B6000E65EFE4F20813181FB01EA5EFE4F8081FF
:101B700090E004C080E090E020E030E0FA013183A2
:101B80002083089580E189BD82E189BD09B400FE0A
:101B9000FDCF8091D8008F7D8093D8008091E000A8
:101BA00082608093E0008091E00081FDFCCF089589
:101BB000CF92DF92EF92FF920F931F93CF93DF9319
:101BC000EC018B016A010E943B0F811133C0C114EB
:101BD000D10439F0F60180819181081B190BC80FDF
:101BE000D91FE12CF12C0115110519F18091E800A4
:101BF00085FD16C08091E8008E778093E800C114BF
:101C0000D10449F0F60180819181E80EF91EF1823C
:101C1000E08285E00FC00E943B0F882321F30AC0B9
:101C200089918093F10001501109FFEFEF1AFF0A2B
:101C3000DACF80E0DF91CF911F910F91FF90EF906D
:101C4000DF90CF9008952091F8013091F901261787
:101C5000370748F06115710539F42091E8002E77B7
:101C60002093E80001C0B90140E061157105A9F1B8
:101C70002091F101222309F443C0253009F442C028
:101C80002091E80023FD40C02091E80022FD32C0F1
:101C90002091E80020FFE9CF4091F3002091F2006D
:101CA00030E0342BFC01CF016115710559F028306B
:101CB000310540F481918093F100615071092F5FEB
:101CC0003F4FF1CF41E02830310509F040E020914D
:101CD000E8002E772093E800C8CF4111C9CF0AC091
:101CE0008091F101882361F0853061F08091E800F6
:101CF00083FD0AC08091E80082FFF2CF80E0089562
:101D000082E0089583E0089581E008952091F8012C
:101D10003091F9012617370748F06115710539F43C
:101D20002091E8002E772093E80001C0B901FC0162
:101D300020E06115710591F18091F101882309F48A
:101D400040C0853009F43FC08091E80083FD3DC06C
:101D50008091E80082FD2FC08091E80080FFE9CFEC
:101D60002091F3008091F20090E0922B61157105B3
:101D700059F08830910540F424912093F100319678
:101D8000615071090196F2CF21E0089709F020E037
:101D90008091E8008E778093E800CBCF2111CCCFE3
:101DA0000AC08091F101882361F0853061F0809153
:101DB000E80083FD0AC08091E80082FFF2CF80E056
:101DC000089582E0089583E0089581E00895982FB2
:101DD000973058F59093E900981739F07091EC001E
:101DE0002091ED005091F00003C0242F762F50E099
:101DF00021FF19C03091EB003E7F3093EB00309112
:101E0000ED003D7F3093ED003091EB003160309379
:101E1000EB007093EC002093ED005093F0002091C4
:101E2000EE0027FF07C09F5FD3CF8F708093E9003C
:101E300081E0089580E008958091F20187FF11C04C
:101E40008091E80082FD05C08091F1018111F8CFF9
:101E500011C08091E8008B770BC08091F10188233D
:101E600049F08091E80080FFF8CF8091E8008E77FC
:101E70008093E80008952091E4003091E50095E614
:101E80004091EC00842F817040FF22C08091E800D7
:101E900080FD1CC08091F101882391F0853091F084
:101EA0008091EB0085FD10C04091E4005091E50069
:101EB0004217530729F39A01915011F784E00895CE
:101EC00082E0089583E0089581E0089580E0089518
:101ED0004091E80042FFDECF08950E94DB0F0E9490
:101EE000E30FE0EEF0E0808181608083E8EDF0E0D8
:101EF00080818F77808319BCA7EDB0E08C918E7FB5
:101F00008C9380818F7E80831092F00108950F93CF
:101F10001F93CF93DF930E94DB0F0E94E30FC8ED66
:101F2000D0E088818F7788838881806888838881E2
:101F30008F7D888319BC1092F1011092ED011092EF
:101F4000EF011092EE0100EE10E0F80180818B7F2E
:101F5000808388818160888342E060E080E00E9425
:101F6000E70EE1EEF0E080818E7F8083E2EEF0E02C
:101F7000808181608083808188608083F801808196
:101F80008E7F8083888180618883DF91CF911F91CC
:101F90000F910895E8EDF0E080818F7E8083E7ED7A
:101FA000F0E080818160808384E082BF81E0809363
:101FB000F0010C94870FE8EDF0E080818E7F808344
:101FC0001092E20008951092DA001092E100089554
:101FD0001F920F920FB60F9211242F933F934F939E
:101FE0005F936F937F938F939F93AF93BF93EF9381
:101FF000FF938091E10082FF0BC08091E20082FF9D
:1020000007C08091E1008B7F8093E1000E944F1216
:102010008091DA0080FF1FC08091D80080FF1BC034
:102020008091DA008E7F8093DA008091D90080FF62
:102030000DC080E189BD82E189BD09B400FEFDCFFC
:1020400081E08093F1010E944A0C05C019BC1092F6
:10205000F1010E94580C8091E10080FF19C080912D
:10206000E20080FF15C08091E2008E7F8093E20045
:102070008091E20080618093E2008091D8008062CC
:102080008093D80019BC85E08093F1010E945C0C1C
:102090008091E10084FF30C08091E20084FF2CC079
:1020A00080E189BD82E189BD09B400FEFDCF809148
:1020B000D8008F7D8093D8008091E1008F7E80933F
:1020C000E1008091E2008F7E8093E2008091E20047
:1020D00081608093E2008091ED01882311F084E01B
:1020E00007C08091E30087FD02C081E001C083E06A
:1020F0008093F1010E945E0C8091E10083FF29C072
:102100008091E20083FF25C08091E100877F80936A
:10211000E10082E08093F1011092ED018091E100F5
:102120008E7F8093E1008091E2008E7F8093E200B9
:102130008091E20080618093E20042E060E080E014
:102140000E94E70E8091F00088608093F0000E946A
:102150005B0CFF91EF91BF91AF919F918F917F9118
:102160006F915F914F913F912F910F900FBE0F9004
:102170001F9018951F920F920FB60F9211242F9354
:102180003F934F935F936F937F938F939F93AF93FF
:10219000BF93CF93DF93EF93FF93C091E900CF708C
:1021A0008091EC00D82FD17080FDD0E81092E9002A
:1021B0008091F000877F8093F00078940E94FE1059
:1021C0001092E9008091F00088608093F000CD2BA0
:1021D000CF70C093E900FF91EF91DF91CF91BF9154
:1021E000AF919F918F917F916F915F914F913F91AF
:1021F0002F910F900FBE0F901F9018951F93CF93A4
:10220000DF93CDB7DEB7AA970FB6F894DEBF0FBE47
:10221000CDBFE2EFF1E088E08E0F9091F100919355
:102220008E13FBCF0E947A0C8091E80083FF1FC1C0
:102230008091F2019091F301492F50E04A3051050D
:1022400008F015C1FA01EA5AFF4F0C94392680387C
:1022500081F0823809F00BC18091F6018F70809374
:10226000E9008091EB0085FB882780F91092E90056
:1022700006C08091EE019091EF01911182609091E2
:10228000E800977F9093E8008093F1001092F100AE
:10229000C8C0282F2D7F09F0EAC0882319F08230AA
:1022A00061F0E5C08091F401813009F0E0C0933025
:1022B00009F080E08093EF012BC08091F40181113F
:1022C00027C08091F6018F7009F4D1C08093E90096
:1022D0002091EB0020FF1CC0933021F48091EB0093
:1022E000806214C09091EB0090619093EB0021E02C
:1022F00030E0A90102C0440F551F8A95E2F74093D0
:10230000EA001092EA008091EB0088608093EB0075
:102310001092E9008091E800877F86C08111A7C0F4
:102320001091F4011F778091E3008078812B8093D6
:10233000E3008091E800877F8093E8000E941C0FF3
:102340008091E80080FFFCCF8091E300806880935B
:10235000E300111102C082E001C083E08093F1012B
:1023600086C08058823008F082C08091F40190913C
:10237000F5018C3D53E0950779F583E08A838AE285
:1023800089834FB7F894DE01139620E03EE051E2D6
:10239000E32FF0E050935700E49120FF03C0E29553
:1023A000EF703F5FEF708E2F90E0EA3010F0C7962D
:1023B00001C0C0968D939D932F5F243149F74FBF85
:1023C0008091E800877F8093E8006AE270E0CE01A8
:1023D00001960E94230E14C0AE014F5F5F4F6091C3
:1023E000F6010E946A0DBC01009709F440C090916B
:1023F000E800977F9093E80089819A810E94860E79
:102400008091E8008B778093E80031C0803879F5BF
:102410008091E800877F8093E8008091ED018093B0
:10242000F1008091E8008E778093E8000E941C0FF5
:102430001EC081111CC09091F4019230C0F48091B3
:10244000E800877F8093E8009093ED010E941C0FC5
:102450008091ED01811106C08091E30087FD02C0EB
:1024600081E001C084E08093F1010E94660C8091BC
:10247000E80083FF0AC08091E800877F8093E8002E
:102480008091EB0080628093EB00AA960FB6F894DF
:10249000DEBF0FBECDBFDF91CF911F91089508958C
:1024A000CF938091F1018823A1F0C091E900CF7012
:1024B0009091EC00892F817090FD80E8C82B1092DC
:1024C000E9008091E80083FD0E94FE10CF70C09368
:1024D000E900CF9108959093750180937401089558
:1024E000E0917401F0917501309721F00190F08135
:1024F000E02D099480E00895E0917401F091750158
:10250000309721F00280F381E02D09940895E09145
:102510007401F0917501309721F00480F581E02D70
:1025200009940895209172013091730182179307E5
:1025300071F09093730180937201E0917401F091B6
:102540007501309721F00680F781E02D09940895F8
:1025500020917001309171018217930771F090936F
:10256000710180937001E0917401F09175013097D1
:1025700021F00084F185E02D0994089508950C94CC
:10258000BE120E94181E0E9434040C94DA1E9F9200
:10259000AF92BF92CF92DF92EF92FF920F931F9371
:1025A000CF93DF9300D000D000D0CDB7DEB70E942C
:1025B0004C040DE010E0AA24A394B12C902E802F9F
:1025C0000E943A05980129583E4F6901F901F080AF
:1025D000F826A1F40150110988F78FEF89838A83C7
:1025E0001B820E94211E8160782F9D838C834981EC
:1025F0005A816B818D810E945E132FC09091DA0108
:1026000091FF04C08E830E9440058E8125E030E05A
:10261000A501022E01C0440F0A94EAF7E42E4F21CF
:10262000C1F029839A828E2191E009F490E09B8386
:102630000E94211E8160782F9D838C8349815A815D
:102640006B818D810E945E13F6018081E826E08215
:1026500004C021503109E0F6BDCF0E94C121109184
:1026600076010E9470121817B9F00E9470128093C0
:10267000760126960FB6F894DEBF0FBECDBFDF9170
:10268000CF911F910F91FF90EF90DF90CF90BF906F
:10269000AF909F900C94690B26960FB6F894DEBF0E
:1026A0000FBECDBFDF91CF911F910F91FF90EF90A3
:1026B000DF90CF90BF90AF909F900895CF93DF931E
:1026C000CDB7DEB72B970FB6F894DEBF0FBECDBFE8
:1026D0004F83588769877A878B87DE01119686E05A
:1026E000FD0111928A95E9F785E0FE013796019088
:1026F0000D928A95E1F749815A816B817C818D81A8
:102700009E810E94A7192B960FB6F894DEBF0FBECC
:10271000CDBFDF91CF910895CF93882309F4C2C034
:10272000C82F823859F40E94701281FDBBC089E322
:102730000E94811C0E944E1D89E30CC0833879F4ED
:102740000E94701280FDAEC083E50E94811C0E9431
:102750004E1D83E50E94C31CCF910C944E1D8438FE
:1027600059F40E94701282FD9DC087E40E94811C72
:102770000E944E1D87E4EECF8CEF8C0F813A48F417
:102780008C2F0E94042481118DC08C2F0E94811CEB
:10279000E3CF80E28C0F883048F4C77081E001C03D
:1027A000880FCA95EAF70E94071DD6CF8BE58C0FDC
:1027B000833078F4C53A29F0C63A31F083E890E0E6
:1027C00005C081E890E002C082E890E0CF910C94CF
:1027D000921288E58C0F833108F064C0C83A39F151
:1027E000C93A41F1CA3A49F1CB3A51F1CC3A59F1DF
:1027F000CD3A61F1C03B69F1CE3A71F1CF3A79F14E
:10280000C13B81F1C23B89F1C33B91F1C43B99F1DA
:10281000C53BA1F1C63BA9F1C73BB1F1C83BB9F13A
:10282000C93BC1F1CA3BC9F180E090E038C082EEFB
:1028300090E035C089EE90E032C08AEE90E02FC083
:1028400085EB90E02CC086EB90E029C087EB90E010
:1028500026C08CEC90E023C08DEC90E020C083E893
:1028600091E01DC08AE891E01AC082E991E017C0AA
:1028700084E991E014C081E292E011C083E292E029
:102880000EC084E292E00BC085E292E008C086E2CE
:1028900092E005C087E292E002C08AE292E0CF9126
:1028A0000C94A812CF910895882309F44BC0823864
:1028B00059F40E94701281FF45C089E30E94811C77
:1028C0000E944E1D89E30CC0833871F40E9470127F
:1028D00080FF38C083E50E94811C0E944E1D83E565
:1028E0000E94C31C0C944E1D843859F40E9470122F
:1028F00082FF28C087E40E94811C0E944E1D87E44D
:10290000EFCF9CEF980F913A58F390E2980F9830E0
:1029100050F4877091E001C0990F8A95EAF7892FEA
:102920000E940D1DDFCF9BE5980F933020F480E0CF
:1029300090E00C949212885A833120F480E090E069
:102940000C94A8120895882321F00E94071D0C946E
:102950004E1D0895882321F00E940D1D0C944E1DDC
:1029600008957F928F929F92AF92BF92CF92DF9203
:10297000EF92FF920F931F93CF93DF931F92CDB7E8
:10298000DEB77C01C62E772EFC01058102950F7003
:10299000128111110E94241D0E947A1C882379F053
:1029A000112369F080E28C0D883048F082E00E94AB
:1029B000631C0E947A1C91E0D82ED92601C0D12C2C
:1029C000E72DE295EF70F0E0E05AFF4F0C943926C6
:1029D000872D807F072D0F70882311F00295007FCF
:1029E000112389F0002309F490C180E28C0D883016
:1029F00020F4802F0E94071D03C0802F0E94171D06
:102A00000E944E1D82C18C2D0E945414002309F493
:102A100095C180E28C0D883020F4802F0E940D1D1E
:102A200003C0802F0E941D1D0E944E1D87C1972D3F
:102A3000907F872D8F70903211F08295807FCC200F
:102A400021F0F1E0CF16B1F01EC0112349F00023B0
:102A500009F414C1013009F011C10E94371D6EC183
:102A6000002319F0013009F469C189830E943A1DDD
:102A700089810AC1112321F0023008F05FC1FEC034
:102A800001115CC101C1112321F0002309F4F6C03A
:102A90003CC1002309F4F8C03EC1872D8695869578
:102AA000837090E0009719F0019761F047C11123FE
:102AB00021F08C2D972D937002C080E090E00E9451
:102AC00092123CC1112321F08C2D972D937002C0DE
:102AD00080E090E00E94A81231C18C2D112319F0E2
:102AE0000E94C92002C00E9431210E94B62126C145
:102AF000872D837009F052C0111120C18C2D829551
:102B000086958770880F880F9C2D9F70892E912C39
:102B1000A12CB12C082E04C0880C991CAA1CBB1C2B
:102B20000A94D2F7C4FE14C00FE010E020E030E0B9
:102B3000B901A80104C0440F551F661F771F8A956D
:102B4000D2F7CB01BA01609570958095909503C03E
:102B500060E070E0CB01272D26952695237030E0AC
:102B60002230310569F02330310589F0682979294F
:102B70008A299B292130310571F00E94EF1ADEC0AD
:102B8000682979298A299B290E940B1BD7C00E949A
:102B9000EF1AC501B4010E94D31AD0C0112319F055
:102BA000872D817001C08695882309F4C7C08C2DBC
:102BB000829586958770880F880F9C2D9F70892E2F
:102BC000912CA12CB12C082E04C0880C991CAA1C95
:102BD000BB1C0A94D2F7C4FE14C00FE010E020E042
:102BE00030E0B901A80104C0440F551F661F771FCC
:102BF0008A95D2F7CB01BA01609570958095909532
:102C000003C060E070E0CB01272D26952695237048
:102C1000422F50E04230510569F04330510589F0B0
:102C2000682979298A299B294130510571F00E9430
:102C3000C91B84C0682979298A299B290E94E51B20
:102C40007DC00E94C91BC501B4010E94AD1B76C0A6
:102C50008C2D90E0FC01E05EF109E531F10508F012
:102C600050C0E059FF4F0C9439260C2D0F70872D62
:102C70008F71112331F00E94461B802F0E94A314F4
:102C80005DC00E94671B802F0E94AA1457C01123A9
:102C900039F0011153C0872D8F710E948C1B4EC0DB
:102CA000023008F04BC0F7CF112339F0872D8F7118
:102CB0000E94461B43C01123C9F3872D8F710E94C8
:102CC000671B3CC0112329F0872D8F710E94311B97
:102CD00035C00E94271B32C0112351F0172D1F71E0
:102CE000812F0E94461B63E0812F0E945A1C26C040
:102CF00081E00E94631C023008F182E00E94631CA4
:102D00001DC0112331F0002389F28C2D0E948C13F9
:102D100015C0002391F28C2D0E9454140FC0472D32
:102D20004F706C2DC7010E9416060E944B1A06C0F8
:102D3000472D4F706C2DC7010E947808DD20F9F0F7
:102D40000E94561C80FD1BC0F70112820E94501C7D
:102D50000E94461BC7010E94CE160E94501C0F9075
:102D6000DF91CF911F910F91FF90EF90DF90CF9067
:102D7000BF90AF909F908F907F900C94671B0F90A7
:102D8000DF91CF911F910F91FF90EF90DF90CF9047
:102D9000BF90AF909F908F907F9008950F931F9357
:102DA000CF93DF93EC01888199812B813C81232B88
:102DB000B9F09F3F11F48F3F99F0CE010E94D007E8
:102DC000882371F0688179818A810E944C1C8C0172
:102DD0000E94011C0E94C81AB801CE010E94B114C1
:102DE000DF91CF911F910F9108950E94241D0E94A1
:102DF000341D0E94F91C0E944E1D0E9467220E94F1
:102E0000B62180E090E00E94921280E090E00C9465
:102E1000A8120E94141D0C94F5160E94411C292F23
:102E200022952F7030E02C3031054CF42A303105DA
:102E30006CF42250310922303105A8F407C02C303F
:102E4000310569F02F30310551F00DC0803F69F038
:102E500018F4803E40F409C0843F29F406C093FB77
:102E6000882780F9089580E0089581E00895CF9340
:102E7000DF9300D000D01F92CDB7DEB70F900F9038
:102E80000F900F900F90DF91CF910895CF93DF9324
:102E900000D000D000D0CDB7DEB726960FB6F8949C
:102EA000DEBF0FBECDBFDF91CF9108951F93CF93AB
:102EB000DF93C091850116E080918601C81799F0D3
:102EC000D0E01C9FF0011D9FF00D1124E957FE4F2B
:102ED0004081518162817381848195810E9446176E
:102EE0002196C770E9CFDF91CF911F91089540914E
:102EF000B7015091B8016091B9017091BA01809108
:102F0000BB019091BC010C9446178091BC01829545
:102F10008F7009F054C08091B901882309F44FC023
:102F200080918501A09186016091B7017091B801EF
:102F30004091BA015091BB01B6E08A1709F43FC035
:102F400090E041155105C1F17F3F11F46F3FA1F1B0
:102F5000B89FF001B99FF00D1124E957FE4F218170
:102F600072132AC02081621327C02281211124C03C
:102F7000238134812417350710F421503109241B93
:102F8000350B283C3105C0F42091BC012F70206125
:102F90002093BC0126E0289FF001299FF00D112409
:102FA000E457FE4F80818F708061808387EB91E0D2
:102FB0000E94CE160C94561701968770BECF0895C6
:102FC000CF92DF92EF92FF920F931F93CF93DF93F5
:102FD000CDB7DEB762970FB6F894DEBF0FBECDBF98
:102FE0008C0185E0F801DE011D9601900D928A9515
:102FF000E1F7D8014C9111965C91119712966C9162
:1030000012971396CD90DC9014973091B701709180
:10301000B8018091BA019091BB01009709F46BC18E
:103020007F3F19F43F3F09F466C1E090B901EE20FB
:1030300009F4C0C02091BC01C816D90628F0F601D9
:10304000E81BF90BCF0104C0809590958C0D9D1D58
:10305000FF24F394883C910578F0F12C207F09F04F
:10306000C6C07C2DD98AC88A89890E94371787EB08
:1030700091E00E94CE16B1C0822F807F09F046C039
:10308000751314C0341312C0611110C02F70206169
:103090002093BC010E94771787EB91E00E94CE1627
:1030A0008091BC01D80115968C932EC0CD2819F1C2
:1030B0005F3F11F44F3FF9F0F62E61111CC0809173
:1030C00085012091860136E0821709F45AC090E00C
:1030D000389FF001399FF00D1124E957FE4F71819F
:1030E000571306C07081471303C07281711103C06A
:1030F00001968770E9CFF62E662309F418C18091F6
:10310000BC0181608093BC01F12C11C1751308C012
:10311000341306C0611104C08091BC01D801C3C042
:103120004D875E878D859E856A8B0E940D176A8903
:103130008823E1F16623D1F12091BC01822F829591
:103140008F7090E0029774F08091B7019091B80170
:1031500098878F831986DB86CA862C87CE010796CF
:103160000E94CE1686E0F801A7EBB1E001900D9227
:103170008A95E1F70E9485170E947717FF24F39440
:10318000D6C04D875E878D859E850E94411C292F64
:1031900022952F7030E0223031050CF0BCC09F70BA
:1031A00009F0B6C0805E883008F4C1C0C8010E9432
:1031B000CE16E4CFC816D90608F453C0F601E81BB2
:1031C000F90BCF01883C910508F450C0F12C7C2DFF
:1031D000D98AC88A89890E943717E7EBF1E086E02F
:1031E000DF011D928A95E9F70E947717A0C0751339
:1031F00014C0341312C0611110C08091BC01F801D9
:103200008583C8010E94CE1686E0E7EBF1E0DF017E
:103210001D928A95E9F7FE2C8AC04D875E878D85C1
:103220009E856A8B0E940D176A89882309F4BECF98
:10323000662309F4BBCF2091BC01822F82958F7049
:1032400090E002970CF48ECF8091B7019091B80175
:103250009A8389831B82DD82CC822E83CE010196E4
:103260007FCF809590958C0D9D1DACCFF62E66235B
:1032700009F49CCF75132EC034132CC02091BC01CF
:1032800020FD1FC0822F82958F70D9F0D80115962E
:103290002C9315978F3049F08F5F982F9295907FE0
:1032A000822F8F70892B15968C93C8010E94CE16A1
:1032B00086E0F801A7EBB1E001900D928A95E1F765
:1032C00093CF86E0F801A7EBB1E001900D928A95CB
:1032D000E1F72DC04D875E878D859E850E940D1775
:1032E000811140CF8091BC0181608093BC01C801F5
:1032F0000E94CE161CC0662309F458CF4D875E8706
:103300008D859E850E940D17882309F44FCF2ACF03
:10331000811148CF0CC0243031050CF047CF9F708D
:1033200009F440CFF8019581907F09F03BCF8F2DB4
:1033300062960FB6F894DEBF0FBECDBFDF91CF917E
:103340001F910F91FF90EF90DF90CF9008951F9302
:10335000CF93DF93CDB7DEB72C970FB6F894DEBFCF
:103360000FBECDBF4F83588769877A878B879C872D
:10337000CE0107960E94E017882369F08F81988517
:103380002A853B85232BF1F19F3F09F063C08F3FD6
:1033900009F060C037C086E0FE013796DE01119665
:1033A00001900D928A95E1F76F817885EA85FB851A
:1033B000309741F17F3F11F46F3F21F12091860159
:1033C00030E0C9010196877099274091850150E04E
:1033D0008417950709F447C069837A83FD83EC83DA
:1033E00096E0929FD001939FB00D1124A957BE4F34
:1033F000FE01319601900D929A95E1F78093860136
:103400000E94561716E080918501909186018917D8
:10341000C1F1189FC001112489579E4F0E94E017E7
:10342000882379F1E09185011E9FF0011124E9576D
:10343000FE4F4081518162817381848195810E9418
:1034400046178091850190E00196877099278093B7
:103450008501D9CF4F81588569857A858B859C8573
:103460000E944617CFCF0E94091710928601109232
:103470008501E7EBF1E086E0DF011D928A95E9F72F
:10348000C1CF2C960FB6F894DEBF0FBECDBFDF9133
:10349000CF911F910895EF92FF920F931F93CF93B7
:1034A000DF938C01009709F46CC0F12CEE24E394B7
:1034B000E8012196F8018491843740F4843008F0C3
:1034C00051C0813081F0823019F15BC0853709F439
:1034D00044C0A8F19CE7980F903708F052C08F774E
:1034E0000E94541441C00E5F1F4FFE01C49180E240
:1034F0008C0F883048F4C7708E2D01C0880FCA9594
:10350000EAF70E94271D14C08C2F0E948C132DC037
:103510000E5F1F4FFE01C49180E28C0F883058F47B
:10352000C7708E2D01C0880FCA95EAF70E942D1D25
:103530000E944E1D1AC08C2F0E94541416C00E5F9C
:103540001F4FFE01C491CC2381F08FE99FE00197CA
:10355000F1F700C00000C150F6CF0E5F1F4FFE0113
:10356000F49003C00E948C138E018F2D882309F4E0
:103570009FCFEFE9FFE03197F1F700C000008150E5
:10358000F5CFDF91CF911F910F91FF90EF900895AC
:1035900008956093C1017093C2018093C301909319
:1035A000C4010C94F5160F931F930091C101109163
:1035B000C2012091C3013091C401DC01CB01802BF9
:1035C000912BA22BB32B8093C1019093C201A093A6
:1035D000C301B093C4011F910F910C94F5160F9382
:1035E0001F930091C1011091C2012091C30130913C
:1035F000C401DC01CB0180239123A223B323809358
:10360000C1019093C201A093C301B093C4011F9163
:103610000F910C94F5160F931F930091C101109117
:10362000C2012091C3013091C401DC01CB0180278C
:103630009127A227B3278093C1019093C201A09341
:10364000C301B093C4011F910F910C94F516109211
:10365000BD011092BE011092BF011092C0010C94E6
:10366000F51641E050E060E070E004C0440F551FE3
:10367000661F771F8A95D2F74093BD015093BE0114
:103680006093BF017093C0010C94F51641E050E0C7
:1036900060E070E004C0440F551F661F771F8A95D5
:1036A000D2F78091BD019091BE01A091BF01B09170
:1036B000C001482B592B6A2B7B2B4093BD015093A3
:1036C000BE016093BF017093C0010C94F51641E0F8
:1036D00050E060E070E004C0440F551F661F771F84
:1036E0008A95D2F740955095609570958091BD016F
:1036F0009091BE01A091BF01B091C0014823592310
:103700006A237B234093BD015093BE016093BF01A8
:103710007093C0010C94F51641E050E060E070E059
:1037200004C0440F551F661F771F8A95D2F78091FA
:10373000BD019091BE01A091BF01B091C001482789
:1037400059276A277B274093BD015093BE016093A0
:10375000BF017093C0010C94F5160F931F93009155
:10376000BD011091BE012091BF013091C001DC016B
:10377000CB01802B912BA22BB32B8093BD01909377
:10378000BE01A093BF01B093C0011F910F910C9493
:10379000F5160F931F930091BD011091BE0120916A
:1037A000BF013091C001DC01CB0180239123A22312
:1037B000B3238093BD019093BE01A093BF01B0934A
:1037C000C0011F910F910C94F5160F931F93009158
:1037D000BD011091BE012091BF013091C001DC01FB
:1037E000CB0180279127A227B3278093BD01909317
:1037F000BE01A093BF01B093C0011F910F910C9423
:10380000F5160895CF92DF92EF92FF920F931F93D8
:10381000CF93DF938C01C090C101D090C201E090A2
:10382000C301F090C4018091BD019091BE01A091AF
:10383000BF01B091C001C82AD92AEA2AFB2ACFE1E8
:10384000D0E0D701C6010C2E04C0B695A795979578
:1038500087950A94D2F780FF06C0B8018C2F0E948A
:10386000CE0A019721F4219760F780E001C08C2FE8
:10387000DF91CF911F910F91FF90EF90DF90CF904C
:103880000895CF93DF93EC010E94021CBE010E94B9
:10389000CE0ADF91CF910895CB010E94411C08957B
:1038A0008091C50185958595859508958091C5017F
:1038B0008770089598E0899F90011124262B20930A
:1038C000C5010C94461B2091C501809582238093ED
:1038D000C501982F977069F430E0482F552747FDB0
:1038E00050952417350729F08595859585950C9475
:1038F000671B08959091C501977081E009F480E0FD
:10390000089590910C01992321F090910D0191114E
:1039100009C020910E0130910F01F90132969FEFFD
:1039200040E01FC0982F9695969596959F3050F53C
:10393000E0910E01F0910F01E90FF11D877021E078
:1039400030E0A90102C0440F551F8A95E2F7CA0171
:103950009181892B818308959F3F39F04F5F4E30CD
:1039600041F051915813F8CF0DC05111F7CF942F5A
:10397000F5CF9F3F39F0F901E90FF11D97FDFA9559
:1039800082830895089590910C01992321F09091DC
:103990000D01911109C020910E0130910F01F90123
:1039A0003296205F3F4F1FC0982F9695969596951B
:1039B0009F30F0F4E0910E01F0910F01E90FF11D3D
:1039C000877021E030E0A90102C0440F551F8A959D
:1039D000E2F7CA0180959181892381830895319608
:1039E000E217F30729F090819813F9CF1082F7CFEF
:1039F000089581E090E0E0910E01F0910F01E80F51
:103A0000F91F1082019680319105A9F708959091D0
:103A1000D901892B8093D901089580959091D9017E
:103A200089238093D90108951092D9010895909126
:103A3000D801892B8093D801089580959091D80161
:103A400089238093D80108951092D8010895909108
:103A5000D701892B8093D701089580959091D70144
:103A600089238093D70108951092D70108958093F8
:103A7000C60108951092C601089580910E0190919B
:103A80000F01FC0131969C01205F3F4F80E0919136
:103A900091118F5FE217F307D1F70895E0910E01BE
:103AA000F0910F018091D9018083E0910E01F09196
:103AB0000F0190818091D801892B8083E0910E01C4
:103AC000F0910F0190818091D701892B80838091A3
:103AD000C601882361F0E0910E01F0910F01908101
:103AE000892B80830E943D1D81111092C601809117
:103AF0000E0190910F010C947C1220E0009739F098
:103B0000AC0141505109842395232F5FF7CF822FB9
:103B10000895CF92DF92EF92FF926C01EE24FF2482
:103B2000C114D104E104F10421F0C701B60120E180
:103B300001C020E0C72ED82EE92EFF24C114D104E5
:103B4000E104F10419F0285FC701B6016B017C01A3
:103B500054E0F694E794D794C7945A95D1F7C114DA
:103B6000D104E104F10419F02C5FC701B6016B0127
:103B70007C0142E0F694E794D794C7944A95D1F734
:103B8000C114D104E104F10419F02E5FC701B6019C
:103B9000DC01CB01B695A79597958795892B8A2B44
:103BA0008B2B09F02F5F822FFF90EF90DF90CF904B
:103BB00008958091F101843021F11092DB0120E41D
:103BC00088E190E00FB6F894A895809360000FBE4E
:103BD0002093600080E00E94690B83B7817F84603E
:103BE00083BF83B7816083BF7894889583B78E7FC6
:103BF00083BF88E10FB6F894809360001092600054
:103C00000FBE0895089508950E94021E0E944C045C
:103C10000E94031E0E94410591E0811101C090E0C5
:103C2000892F08950E9409170E9470120C94690B45
:103C300082E084BD93E095BD9AEF97BD80936E00BE
:103C400008952FB7F8948091DC019091DD01A09147
:103C5000DE01B091DF012FBF0895CF92DF92EF9286
:103C6000FF920F931F932FB7F8944091DC0150916E
:103C7000DD016091DE017091DF012FBF6A017B01E0
:103C8000EE24FF248C0120E030E0C016D106E206CD
:103C9000F30610F4415051099A01281B390BC90150
:103CA0001F910F91FF90EF90DF90CF9008951F929A
:103CB0000F920FB60F9211248F939F93AF93BF93E0
:103CC0008091DC019091DD01A091DE01B091DF01D6
:103CD0000196A11DB11D8093DC019093DD01A0939D
:103CE000DE01B093DF01BF91AF919F918F910F9053
:103CF0000FBE0F901F9018950E946D0FF8942FEF34
:103D000087EA91E6215080409040E1F700C0000032
:103D100087E090EBDC018093FB019093FC01A09382
:103D2000FD01B093FE019CE088E10FB6F894A895E0
:103D3000809360000FBE90936000FFCFEF92FF92E0
:103D40000F931F93CF93DF93D82FCDE08C2F0E943A
:103D50003A0505E010E0E82EF12CC701002E02C064
:103D6000959587950A94E2F780FF09C0602F7C2F14
:103D700080E00E947908D81302C081E006C001509B
:103D8000110958F7C15010F780E0DF91CF911F91D2
:103D90000F91FF90EF900895CF93C82F8CE20E946F
:103DA0009E1E882321F08C2FCF910C949E1E80E0C4
:103DB000CF910895CF930E942120811102C00E94CB
:103DC0000720C5E6C15049F00E944C048FE39CE9EE
:103DD0000197F1F700C00000F5CF89E20E94CC1EE8
:103DE000811113C18AE20E94CC1E81110E9407201A
:103DF00085E00E94CC1E81110E947C1E0E942C2016
:103E00008093DA0187E00E94CC1E8823A9F18BE120
:103E10000E94CC1E882351F08091DA0181FB222779
:103E200020F991E0922790FB81F90EC08EE00E946C
:103E3000CC1E882361F08091DA0182FB222720F9D1
:103E400091E0922790FB82F98093DA0115C080E11E
:103E50000E94CC1E9091DA01882341F093FB222727
:103E600020F981E0822780FB93F904C0892F809597
:103E700080FB90F99093DA018091DA010E94302062
:103E80000E943E208093FA0180EE0E94CC1E88237F
:103E900041F08091FA01982F909590FB80F98093E2
:103EA000FA0189E30E94CC1E882359F08091FA011F
:103EB00081FB222720F991E0922790FB81F98093E2
:103EC000FA0182EE0E94CC1E882359F08091FA01FB
:103ED00082FB222720F991E0922790FB82F98093C0
:103EE000FA0186EE0E94CC1E882359F08091FA01D7
:103EF00083FB222720F991E0922790FB83F980939E
:103F0000FA0183EE0E94CC1E882359F08091FA01B9
:103F100084FB222720F991E0922790FB84F980937B
:103F2000FA0185E30E94CC1E882359F08091FA01A2
:103F300085FB222720F991E0922790FB85F9809359
:103F4000FA0181E30E94CC1E882359F08091FA0186
:103F500086FB222720F991E0922790FB86F9809337
:103F6000FA0181E10E94CC1E882359F08091FA0168
:103F700087FB222720F991E0922790FB87F9809315
:103F8000FA018091FA010E9442208091FA0187FB98
:103F9000882780F980930D0187E20E94CC1EC82FEC
:103FA0008EE10E94CC1E8111C2608FE10E94CC1E66
:103FB0008111C46080E20E94CC1E8111C86081E240
:103FC0000E94CC1E8111C06182E20E94CC1E811130
:103FD000C06283E20E94CC1E8111C06484E20E9410
:103FE000CC1E882311F0C06802C0CC2329F08C2F8E
:103FF0000E9439206C2F03C00E943520682F70E08A
:1040000080E090E0CF910C94C91ACF9108956DEEA5
:104010007EEF80E090E00E94732660E082E090E016
:104020000E94612660E083E090E00E94612660E0EB
:1040300084E090E00E94612660E085E090E00C94CE
:10404000612680E090E00E945B2621E08D3E9E4F3D
:1040500009F020E0822F089582E090E00C9453262E
:10406000682F82E090E00C94612683E090E00C944D
:104070005326682F83E090E00C94612684E090E062
:104080000C945326682F84E090E00C946126809174
:10409000E20180FF0BC06091130185E0689FB001D1
:1040A000112475956795759567952BC081FF09C09B
:1040B0006091130185E0689FB001112475956795A3
:1040C00020C082FF07C06091130185E0689FB001A6
:1040D000112417C09091E3019923D1F0609112014E
:1040E000961788F72091130185E0289F90011124ED
:1040F000929FA001939F500D112470E0CA010E946D
:1041000025266038710540F46115710539F002C04B
:1041100065E070E0862F08958FE7089581E00895A7
:104120008091E20180FF08C06091110170E07595F7
:1041300067957595679521C081FF06C06091110153
:1041400070E07595679519C082FF04C060911101F8
:1041500070E010C09091E3019923C1F060911001CB
:104160009617A0F780911101899FC001112470E07A
:104170000E9425266038710528F46115710521F02B
:10418000862F08958FE7089581E0089561E070E03B
:10419000F4CF803F21F40E944720819504C0813FE5
:1041A00029F40E9447208093E6010895823F21F47C
:1041B0000E944720819504C0833F29F40E94472034
:1041C0008093E5010895893F19F40E94902005C06D
:1041D0008A3F31F40E94902081958093E7010895F1
:1041E0008B3F21F40E949020819504C08C3F29F4DC
:1041F0000E9490208093E8010895843F21F48091EB
:10420000E401816017C0853F21F48091E401826060
:1042100011C0863F21F48091E40184600BC0873F88
:1042200021F48091E401886005C0883F31F48091D9
:10423000E40180618093E40108958D3F21F4809131
:10424000E20181600BC08E3F21F48091E201826027
:1042500005C08F3F29F48091E20184608093E201E0
:104260000895803F39F48091E60187FF6CC0109279
:10427000E60169C0813F29F48091E6011816BCF37C
:1042800062C09091E501823F29F497FF5CC01092D3
:10429000E50159C0833F19F41916CCF354C0893F86
:1042A00041F48091E70118160CF04DC01092E7011F
:1042B0004AC08A3F29F48091E70187FF44C0F6CFC6
:1042C0008B3F39F48091E80187FF3DC01092E801EF
:1042D0003AC08C3F29F48091E8011816BCF333C032
:1042E000843F21F48091E4018E7F17C0853F21F443
:1042F0008091E4018D7F11C0863F21F48091E4011B
:104300008B7F0BC0873F21F48091E401877F05C03C
:10431000883F31F48091E4018F7E8093E40113C0E3
:104320008D3F21F48091E2018E7F0BC08E3F21F4FE
:104330008091E2018D7F05C08F3F29F48091E201D9
:104340008B7F8093E2018091E50181110EC0809105
:10435000E60181110AC08091E701811106C08091B8
:10436000E801811102C01092E301089584EE91E00A
:104370000E9487120E94211E9093E1018093E00128
:1043800008951F93CF93DF938091E0019091E10115
:104390000E942D1EAC019091E301992321F0209100
:1043A000140130E006C0209115018AE0289F900199
:1043B00011244217530708F486C08091E501C0918B
:1043C000E601D091E7011091E801811107C0C11108
:1043D00076C0D11174C0111172C075C09F3F19F021
:1043E0009F5F9093E301181624F40E944720809366
:1043F000E5018091E50187FF05C00E944720819576
:104400008093E5011C1624F40E9447208093E60166
:104410008091E60187FF05C00E9447208195809327
:10442000E6016091E501662339F1C091E601CC23F4
:1044300019F1772767FD7095872F972F0E943625F2
:1044400023E333E343E35FE30E949A250E940325BD
:104450006093E5016C2F772767FD7095872F972F65
:104460000E94362523E333E343E35FE30E949A256A
:104470000E9403256093E6011D1624F40E949020FB
:104480008093E7018091E70187FF05C00E9490209B
:1044900081958093E701111624F40E949020809367
:1044A000E8018091E80187FF05C00E949020819576
:1044B0008093E801DF91CF911F910C94B6219F3F2B
:1044C00009F08ECF96CFDF91CF911F910895E4EE42
:1044D000F1E085E0DF011D928A95E9F71092E30192
:1044E0001092E2010895833081F128F4813059F06F
:1044F0008230D1F00895853009F449C0B8F1863092
:1045000009F456C0089580911501262F30E0280F38
:10451000311D2F3F310524F4680F60931501089574
:104520008FEF80931501089580911401262F30E0BC
:10453000280F311D2F3F310524F4680F60931401BB
:1045400008958FEF80931401089580911301262F11
:1045500030E0280F311D2F3F310524F4680F6093A0
:10456000130108958FEF8093130108958091120134
:10457000262F30E0280F311D2F3F310524F4680F1E
:104580006093120108958FEF809312010895809136
:104590001101262F30E0280F311D2F3F310524F463
:1045A000680F6093110108958FEF809311010895B2
:1045B00080911001262F30E0280F311D2F3F31054B
:1045C00024F4680F6093100108958FEF8093100119
:1045D0000895833011F128F4813049F0823091F050
:1045E0000895853081F120F18630C1F108958091E0
:1045F0001501681720F4861B809315010895109209
:104600001501089580911401681720F4861B80938A
:1046100014010895109214010895809113016817F0
:1046200020F4861B809313010895109213010895BE
:1046300080911201681720F4861B8093120108955F
:1046400010921201089580911101681720F4861BC1
:104650008093110108951092110108958091100125
:10466000681720F4861B80931001089510921001A2
:1046700008950F931F938D3109F46BC008F03FC06C
:104680008E3009F47FC0C0F4873009F469C068F443
:10469000863009F0B1C08091DA01817F8E7F8093EE
:1046A000DA0181E08093EA01A8C0883009F4A2C051
:1046B0008B3009F49FC0A0C0863109F49BC078F408
:1046C000803109F472C0813109F096C00E94091747
:1046D00090910D0181E0892780930D018BC0893174
:1046E00009F488C08B3109F087C08091DA0181FB21
:1046F000222720F991E0922790FB81F94CC0853365
:1047000009F470C048F4873209F46CC008F459C049
:10471000893209F467C070C0833438F48A3308F0F2
:104720004EC0883309F466C067C0833409F45AC0A8
:10473000883409F061C00E9409170FEF13ED20E3E0
:10474000015010402040E1F700C000000E947C1E94
:1047500051C00E94BD240E9470120E94690B4AC081
:104760009091DA01892F8095817080FB90F929F072
:10477000966098609093DA0140C0997F977F9093FC
:10478000DA0138C08091DA0182FB222720F991E01A
:10479000922790FB82F98093DA01992359F1809155
:1047A000DA0181608093DA0125C08091DA0183FB10
:1047B000222720F991E0922790FB83F9ECCF8953CF
:1047C00001C08D5141E050E060E070E08A019B0142
:1047D00004C0000F111F221F331F8A95D2F7C90191
:1047E000B80104C061E070E080E090E00E94C91A66
:1047F0000E94091781E001C080E01F910F91089588
:1048000080E0089580E00895CF93C82F8091EA0159
:10481000813079F018F08230E9F187C0E0910E0123
:10482000F0910F018081813169F0823209F07FC0FF
:1048300009C0E0910E01F0910F018081813111F0EA
:10484000823261F48C2F0E940024811104C08C2FCD
:104850000E9439231DC081E090E01AC08C2F0E9475
:104860000224811114C0C43179F048F4CB3079F0BE
:10487000C03109F060C082E08093EA0108C0C9320B
:1048800019F0C83321F057C01092EA0154C081E0FA
:10489000817053C0C93289F118F5C43171F1A8F49F
:1048A000C73009F046C08AE08093150194E19093E7
:1048B000140193E0909313018093120188E0809398
:1048C000110188E28093100134C0CE51C63088F5C2
:1048D000EC2FF0E0E65DFE4F80818093E90129C076
:1048E000CE34E9F020F4CB3421F56AE013C0C135B1
:1048F00079F0C235F1F461E00DC08091E9018823BF
:1049000019F01092E90115C081E08093EA0115C009
:1049100061E006C08091E9010E9473220AC06AE04A
:104920008091E9010E94E92204C01092EA0180E02E
:1049300004C081E002C080E0ABCFCF910895E1E8F0
:10494000F0E08081886080838081816080838FB780
:10495000F89493E09093890090ED909388008FBF36
:104960000895EFE6F0E08081826080830895EFE6AD
:10497000F0E080818D7F80830895EFE6F0E0908104
:1049800082E08927808308951F920F920FB60F92BD
:1049900011242F933F934F935F936F937F938F9344
:1049A0009F93AF93BF93EF93FF938091EB0190910F
:1049B000EC0101969093EC018093EB01811103C00F
:1049C00082E00E94690BE091EC01E695E695F0E04B
:1049D000EB54F94FE4918091EB018E1303C080E01A
:1049E0000E94690BFF91EF91BF91AF919F918F91C1
:1049F0007F916F915F914F913F912F910F900FBEDB
:104A00000F901F90189504D06894B1118DC008952F
:104A100070D088F09F5790F0B92F9927B751A0F028
:104A2000D1F0660F771F881F991F1AF0BA95C9F742
:104A300012C0B13081F077D0B1E0089574C0672F13
:104A4000782F8827B85F39F0B93FCCF386957795F2
:104A50006795B395D9F73EF49095809570956195DB
:104A60007F4F8F4F9F4F0895E89409C097FB3EF406
:104A700090958095709561957F4F8F4F9F4F9923AB
:104A8000A9F0F92F96E9BB279395F6958795779529
:104A90006795B795F111F8CFFAF4BB0F11F460FFE9
:104AA0001BC06F5F7F4F8F4F9F4F16C0882311F041
:104AB00096E911C0772321F09EE8872F762F05C055
:104AC000662371F096E8862F70E060E02AF09A95F0
:104AD000660F771F881FDAF7880F9695879597F9E5
:104AE000089557FD9058440F551F59F05F3F71F0DE
:104AF0004795880F97FB991F61F09F3F79F0879545
:104B00000895121613061406551FF2CF4695F1DFCD
:104B100008C0161617061806991FF1CF869571055D
:104B2000610508940895E894BB2766277727CB0191
:104B300097F908950BD078C069D028F06ED018F09E
:104B4000952309F05AC05FC01124EECFCADFA0F34D
:104B5000959FD1F3950F50E0551F629FF001729F12
:104B6000BB27F00DB11D639FAA27F00DB11DAA1F31
:104B7000649F6627B00DA11D661F829F2227B00D7E
:104B8000A11D621F739FB00DA11D621F839FA00D09
:104B9000611D221F749F3327A00D611D231F849F59
:104BA000600D211D822F762F6A2F11249F575040B0
:104BB0008AF0E1F088234AF0EE0FFF1FBB1F661F4B
:104BC000771F881F91505040A9F79E3F510570F004
:104BD00014C0AACF5F3FECF3983EDCF3869577953F
:104BE0006795B795F795E7959F5FC1F7FE2B880FFF
:104BF000911D9695879597F9089597F99F6780E895
:104C000070E060E008959FEF80EC089500240A941E
:104C10001616170618060906089500240A94121697
:104C20001306140605060895092E0394000C11F4CA
:104C3000882352F0BB0F40F4BF2B11F460FF04C077
:104C40006F5F7F4F8F4F9F4F089597FB072E16F48E
:104C5000009407D077FD09D00E943F2607FC05D0BD
:104C60003EF4909581959F4F0895709561957F4F83
:104C70000895EE0FFF1F0590F491E02D0994AA1BF3
:104C8000BB1B51E107C0AA1FBB1FA617B70710F037
:104C9000A61BB70B881F991F5A95A9F78095909569
:104CA000BC01CD010895F999FECF92BD81BDF89A5E
:104CB000992780B50895A8E1B0E042E050E00C9457
:104CC0007B26262FF999FECF92BD81BDF89A0197D8
:104CD00000B4021639F01FBA20BD0FB6F894FA9A44
:104CE000F99A0FBE08950196272F0E9462260C9410
:104CF0006126DC01CB01FC01F999FECF06C0F2BDB3
:104D0000E1BDF89A319600B40D9241505040B8F789
:064D10000895F894FFCFA6
:104D160002206B0BF90BD60BA20B6E0B0101C70120
:104D260028080A03140A3F4D363976062906F30584
:104D3600BA054D0566057F059805010203040506BB
:044D46000708090051
:00000001FF
